:020000040800F2
:1000000000040220010200080302000803020008A5
:1000100003020008030200080302000803020008AC
:10002000030200080302000803020008C5270008B5
:10003000030200080302000803020008030200088C
:10004000030200080302000803020008030200087C
:100050000302000803020008DD390008093A00081D
:10006000353A0008613A00088D3A0008030200089A
:10007000030200080302000803020008030200084C
:10008000030200080302000803020008030200083C
:10009000030200080302000803020008B93A00083E
:1000A000030200080302000803020008030200081C
:1000B00001380008030200080302000803020008D8
:1000C00003020008030200080302000803020008FC
:1000D0000302000803020008E9100008FD100008F0
:1000E000213B000803020008030200080302000885
:1000F00003020008030200080302000803020008CC
:1001000003020008030200080302000803020008BB
:1001100003020008030200080302000803020008AB
:10012000030200080302000803020008030200089B
:10013000030200080302000803020008030200088B
:10014000030200080302000803020008312F000820
:10015000030200080302000803020008030200086B
:10016000030200080302000803020008030200085B
:10017000030200080302000803020008030200084B
:10018000030200080302000811110008030200081E
:10019000030200080302000803020008030200082B
:1001A000030200080302000803020008030200081B
:1001B000030200080302000803020008030200080B
:1001C00003020008030200080302000803020008FB
:1001D00003020008030200080302000803020008EB
:1001E00003020008030200080302000803020008DB
:1001F00003020008030200080302000803020008CB
:1002000002E000F000F8FEE772B6394880F3088893
:10021000384880F3098838484EF60851CEF200017C
:10022000086040F20000CCF200004EF63471CEF2CD
:1002300000010860BFF34F8FBFF36F8F40F20000E3
:10024000C0F2F0004EF68851CEF200010860BFF314
:100250004F8FBFF36F8F4FF00000E1EE100A4EF6A4
:100260003C71CEF200010860062080F31488BFF3D1
:100270006F8F02F0E5FA03F04BFA4FF055301F494B
:100280001B4A91423CBF41F8040BFAE71C49194A4A
:1002900091423CBF41F8040BFAE71A491A4A1B4B3A
:1002A0009A423EBF51F8040B42F8040BF8E70020D5
:1002B0001749184A91423CBF41F8040BFAE702F093
:1002C00003FB03F08FFA144C144DAC4203DA54F8DC
:1002D000041B8847F9E700F03FF8114C114DAC4280
:1002E00003DA54F8041B8847F9E702F0EBBA000080
:1002F0000004022000240220000000080000022068
:1003000000040220A83F00080024022050240220FC
:1003100050240220D84102200002000800020008F8
:1003200000020008000200082DE9F04F2DED108AB0
:10033000C1F80CD0D0F80CD0BDEC108ABDE8F08F1D
:10034000002383F311882846A047002001F0DEFE39
:1003500001F08EFE00DFFEE770B5214C6FF07703F1
:10036000002523706FF07F061E236570A570E57071
:1003700025716571A571E57125726672A372E572CA
:1003800000F03CFD20B10E2325726672A372E57267
:1003900002F0EEF9044602F00FFA0546D8B9114B07
:1003A0009C421AD001339C4218BF054641F2883462
:1003B00004BF01250024002002F0E0F90DB100F097
:1003C000B7F800F08DFD00F06BFC204600F050F90E
:1003D00000F0AEF8F9E70024EDE70446EBE700BFD4
:1003E00050240220010007B008B500F0D7FBA0F1AF
:1003F00020035842584108BD07B5054B02211B8810
:10040000ADF8043001A800F035FC03B05DF804FB42
:10041000203C0008064991F8243033B1002308221B
:10042000086A81F8243000F05FBC0120704700BFEB
:10043000702402202DE9F84F234C94F8243005460F
:10044000884617468BBB2E46DFF87C90002F38D0AD
:1004500094F824A0BAF1000F05D12022FF214846CC
:10046000266200F02BFDCAF10805BD4228BF3D46BB
:100470005FFA85FBAD0041462A4604EB8A0000F096
:10048000F3FC94F82430A7EB0B079B445FFA8BFB3B
:10049000BBF1080F2E44A844FFB284F824B0D5D194
:1004A000FFF7B8FF0028D1D108E0266A06EB8306E3
:1004B000B042C9D0FFF7AEFF0028C4D10020BDE88C
:1004C000F88F0120BDE8F88F7024022010B520239A
:1004D00083F311881248C3680BB101F09DFE00231D
:1004E000104A0F484FF47A7101F05AFE002383F34B
:1004F00011880D4C236813B12368013B23606368A6
:1005000013B16368013B6360084B1B7833B96368C0
:1005100023B9022000F09EFC3223636010BD00BFAF
:100520005C240220CD040008A02902209824022087
:100530002DE9F041444B454953F8042F013201D1D4
:10054000BDE8F0818B42F7D1414C424B22689A4280
:1005500078D9414B9B6803F1006303F5C0339A429D
:1005600070D2002000F0B8FB3C4B0220187000F065
:1005700067FC3B4B1A6C00221A64196E1A66196EDE
:10058000596C5A64596E5A66596E596941F0800126
:100590005961596921F0800159615969196941F01E
:1005A00000511961196921F0005119611B6972B676
:1005B0002C492D4B0B601D682468BFF34F8FBFF390
:1005C0006F8F2A4BC3F88420BFF34F8F5A6922F4F0
:1005D00080325A61BFF34F8FD3F88020C2F3C9062F
:1005E000C2F34E325201B70743F6E07E02EA0E082C
:1005F00038463146013948EA000CB1F1FF3FC3F8F3
:1006000074C200F14040F5D1203A12F1200FEDD133
:10061000BFF34F8FBFF36F8FBFF34F8FBFF36F8F5A
:100620005A6922F400325A610022C3F85022BFF303
:100630004F8FBFF36F8F202383F31188AD4685F36F
:1006400008882047BDE8F081FC7F01081C80010874
:1006500004800108FF7F0108502402209824022012
:100660000038024008ED00E00080010800ED00E0E5
:100670002DE9F04FB04C97B020228146FF210EA803
:10068000A66800F01BFCAD4A1378A346A3B9AC489A
:100690000121C3601170202383F31188C3680BB15B
:1006A00001F0BAFD0023A74AA5484FF47A7101F082
:1006B00077FD002383F31188B9F1000F02D0A24B1C
:1006C000C3F80090A14BA04A00241C70546025463A
:1006D00027469846012000F0B3FBB9F1000F00F067
:1006E0002282994B1B68002B40F01D8217B0BDE899
:1006F000F08F0220FFF778FE002840F00E82944B26
:100700001B88ADF82430022109A800F0B3FAE1E714
:100710004FF47A7000F042FA031E0193EFDB0220DF
:10072000FFF762FE82460028E9D0019B581E04288C
:1007300000F2F581DFE800F0030D1013160016A893
:10074000052340F8343D042100F094FA5446002774
:1007500052E004217848F7E704217E48F4E70421B9
:100760007D48F1E71C24204600F0B8FA04340990D3
:10077000042109A800F07EFA2C2CF4D1E6E7002D24
:10078000BDD0002CBBD00220FFF72EFE054600286E
:1007900000F0C781012000F09FFA022088F80000D5
:1007A00000F04EFB0024E3B21846019300F0A4FAD7
:1007B000824648B1019B184600F0AEFA0134002889
:1007C000F1D12C46654B9BE70123022088F80030CD
:1007D00000F02CFB5646DBF808309E4206D230462D
:1007E00000F07CFA0130ECD10436F4E7564B0026D9
:1007F00088F800605E602C4600F068FB1DB1002C9C
:1008000018BF4FF00009FFF7F7FD63E7002D3FF435
:1008100076AF002C3FF473AF022088F8000000F0A0
:100820000FFB322000F0BAF9B0F1000AC0F2798172
:100830001AF0030540F07581DBF8082006EB0A0387
:10084000934200F26E81BAF5807F00F26A81444BD8
:10085000019355450DDA4FF47A7000F09FF902903C
:10086000029A002AC0F25D81019B029AEA54013586
:10087000EEE7C820FFF7B8FD0546002800F05181DB
:100880001F2E11D8C6F12004544528BF54460EAB84
:1008900026F0030022463249184400F0E5FA2246C9
:1008A000FF212F4800F00AFB4FEAAA0A5FFA8AF2FA
:1008B0002B493046FFF7BEFD0446002881D006EBE9
:1008C0008A06054698E70220FFF78EFD00283FF4D0
:1008D00016AFFFF79FFD00283FF411AF00229246AC
:1008E000DBF808309A4259D21F2A1ED80E9B0133DA
:1008F0001BD022F0030316A90B4453F8203C0993A4
:100900001848436883B3174800210DF1240E11F8ED
:100910000E3083EA0A03DBB2013150F82330042998
:1009200083EA1A2AF3D10432DAE71046019200F082
:10093000D5F9019A0990E3E7502402209C25022072
:100940005C240220CD040008A02902209824022063
:10095000223C00085424022058240220243C000891
:100960009C240220A025022019464FF0080E11F009
:10097000010F4FEA51011FBF81F06D4181F4380131
:1009800081F4034181F02001BEF1010EEFD140F866
:1009900023100133B3F5807FE6D1B4E716A8042114
:1009A00040F84CAD00F066F926E716A8002340F8A1
:1009B000343D642100F02AF900287FF4A0AE022023
:1009C000FFF712FD00283FF49AAE099800F0B6F93F
:1009D00016AB43F8480D04211846E3E716A8002398
:1009E00040F8343D642100F011F900287FF487AE0F
:1009F0000220FFF7F9FC00283FF481AE099800F0CF
:100A0000ABF916AB43F8440DE5E70220FFF7ECFC29
:100A100000283FF474AE00F0A5F916AB43F8400D82
:100A2000D9E70220FFF7E0FC00283FF468AE09A9EF
:100A3000142000F09DF9824616A8042140F83CAD30
:100A400000F018F9514609A8ACE7322000F0A6F8EA
:100A5000B0F1000AFFF653AE1AF0030F7FF44FAE69
:100A6000DBF808200AEB070393423FF648AE02206A
:100A7000FFF7BAFC00283FF442AE2AF0030ABA445A
:100A8000BA453FF4B9AE384600F028F90421089081
:100A900008A800F0EFF80437F2E74FF47A70FFF798
:100AA000A3FC00283FF42BAEFFF7B4FC00283FF472
:100AB00089AE0E9B01330CD008220EA90020FFF74F
:100AC000B9FC00283FF47EAE2022FF210EA800F0E2
:100AD000F5F9FFF791FC304801F01EFB06E616A879
:100AE000002340F8343D642100F090F8824600284D
:100AF0007FF405AE0220FFF777FC00283FF4FFAD3E
:100B0000FFF77AFC41F2883001F006FB099800F00B
:100B100025FAD14600F0DAF9DCE505466CE6002757
:100B2000EDE52546EBE5002000F038F80290029B49
:100B3000002BFFF6D2AD012000F078F9029B213B9B
:100B4000122B3FF6C7AD01A252F823F0F3060008BE
:100B5000110700087F070008D5060008D506000821
:100B6000D50600080D0800084B0A0008C708000851
:100B7000AB090008DD0900080B0A0008D5060008CB
:100B8000230A0008D50600089B0A0008F907000898
:100B9000D5060008DF0A0008A08601002DE9F3470A
:100BA00002AE00244FF47A7506F8014D144FDFF8B9
:100BB0005880454397F900305A1C5FFA84F901D0F8
:100BC000A34212D158F8240003680122D3F820A0D0
:100BD00031462B46D047012807D10A4B9DF8070024
:100BE00083F8009002B0BDE8F0870134042CE1D115
:100BF0004FF4FA7001F090FA4FF0FF30F2E700BFC7
:100C000000240220C4290220303C00082DE9F047CE
:100C10004FF47A75144FDFF8588006464D43002490
:100C200097F900305A1C5FFA84F901D0A34210D121
:100C300058F8240003680422D3F820A031462B463C
:100C4000D047042805D1094B83F800900020BDE867
:100C5000F0870134042CE3D14FF4FA7001F05CFA10
:100C60004FF0FF30BDE8F08700240220C4290220A5
:100C7000303C000830B4074B1A78074B53F8224039
:100C80002368DD69054B0A46AC460146204630BC68
:100C9000604700BFC4290220303C0008A086010044
:100CA000F8B501F071FC094C094E0A4F207000257F
:100CB00030682378834207D901F060FC336805442B
:100CC0000133BD423360F3D9F8BD00BFC52902200E
:100CD000A8290220FF7F010001F014BD00F100608F
:100CE00000F5C0300068704700F10060920000F528
:100CF000C03001F09FBC0000054B1A68054B1B7803
:100D00009B1A834202D9104401F038BC002070477E
:100D1000A8290220C529022038B5074D04462868B5
:100D2000204401F033FC28B928682044BDE838404D
:100D300001F044BC38BD00BFA829022010F0030315
:100D400008D1B0F5806F05D800F10050A0F57120F2
:100D50000068704700207047014BC058704700BFC3
:100D600020F4F01F014B1868704700BF002004E01A
:100D7000F0B5204B1E68204B1F885D6893F9084032
:100D8000C6F30B02BA424FEA164622D09F89BA42F6
:100D900021D01F8BBA4206D102220C2404FB02335D
:100DA0005D6893F90840B6F5805F16D041F2010303
:100DB0009E4208BF5A24421E0A44013D0B469342FC
:100DC00015D215F9016F581C4EB1034600F8016C9D
:100DD000F5E70022E1E70122DFE74124EBE72C25DC
:100DE00082421D7001D9981C5C70401AF0BD1846F3
:100DF000FBE700BF002004E004240220094B5B88CD
:100E0000B3F5805F09D041F20102934207D101227C
:100E1000054B03EB8203D87870470022F8E70020E7
:100E2000704700BF002004E0283C0008022802BFF1
:100E3000024B4FF480529A61704700BF001002408D
:100E4000022802BF024B4FF080529A61704700BFE8
:100E500000100240022801BF024A536983F4805304
:100E6000536170470010024010B50023934203D035
:100E7000CC5CC4540133F9E710BD000030B5441E0A
:100E800014F9010F0B4660B193F90050854201F14E
:100E9000010106D11AB993F90020801A30BD013A38
:100EA000EEE7002AF7D1104630BD000002460346A7
:100EB000981A13F9011B0029FAD17047024403461E
:100EC000934202D003F8011BFAE77047024B1A78ED
:100ED000024B1A70704700BFC42902200024022070
:100EE000F8B5184C1848194D194E174F00F054FC1E
:100EF0002146154800F07CFC23681648DA6ED2F8CB
:100F0000043843F00203C2F8043801F005F9206800
:100F1000114900F07BFD2368DA6ED2F8043823F023
:100F20000203C2F804384FF4E1332B60002456F872
:100F30002400B84202D0294600F08CFB0134042C76
:100F4000F5D1F8BD283D00084C370220AC2902201D
:100F5000303C000840420F00703D000838B50B4B94
:100F60001A780B4B53F822400A4B9C4205460CD092
:100F7000094B002118461822FFF7A0FF0560014623
:100F80002046BDE8384000F065BB38BDC4290220CA
:100F9000303C00084C370220AC290220026843682C
:100FA0001143016003B1184770470000024A1368FB
:100FB00043F0C0031360704700440040024A1368C6
:100FC00043F0C0031360704700480040024A1368B2
:100FD00043F0C00313607047007800402DE9F047EC
:100FE000C66D3768F46934620546200719D014F0DD
:100FF000080F0CBF00218021E20748BF41F020010B
:10100000A30748BF41F04001600748BF41F4807129
:10101000202383F31188281DFFF7C0FF002383F3EB
:101020001188E2050AD5202383F311884FF400715B
:10103000281DFFF7B3FF002383F311884FF0200929
:101040004FF0000A14F0200831D13B0616D54FF0BE
:10105000200905F1380A200610D589F31188504679
:1010600000F06CFA00282FDA0821281DFFF796FF00
:1010700027F080033360002383F3118879060DD5B0
:1010800062060BD5202383F31188EA6C2B6D9A42FC
:1010900001D12B6CEBB9002383F31188E30620D533
:1010A000AA6E1369EBB15069BDE8F047184789F3A0
:1010B0001188736A95F864102846194000F0D8FA30
:1010C0008AF31188F469BDE7B06288F31188F46986
:1010D000C1E71021281D27F04007FFF75FFF3760A9
:1010E000D9E7BDE8F087000008B50348FFF776FFB1
:1010F000BDE8084001F076BBC829022008B50348C6
:10110000FFF76CFFBDE8084001F06CBB342A0220F9
:1011100008B50348FFF762FFBDE8084001F062BB75
:10112000A02A022037B52D4C2D4D204600F086FA1E
:10113000009404F1140000234FF40072294900F0D8
:1011400047F94FF40072009404F13800264B274908
:1011500000F0C0F9264BE3652566264C0B212620BE
:1011600000F0C4F8204600F069FA009404F114007D
:1011700000234FF40072204900F02AF94FF4007266
:10118000009404F138001D4B1D4900F0A3F91D4BDC
:10119000E36525661C4C0B21272000F0A7F82046AC
:1011A00000F04CFA04F11400009400234FF4007294
:1011B000164900F00DF904F138000094144B15495C
:1011C0004FF4007200F086F9134BE3650B215220B7
:1011D000256603B0BDE8304000F088B8C829022079
:1011E00080F937030C2B0220AD0F00080C310220D0
:1011F00000440040342A02200C2D0220BD0F0008BC
:101200000C33022000480040A02A02200C2F0220AC
:10121000CD0F00080C350220007800402E4B00292D
:1012200008BF1946037C8166012B30B50CD12B4BCE
:10123000984235D12A4B1A6C42F400321A641A6E65
:1012400042F400321A661B6E0A68036EC46D03EB2B
:101250005203B3FBF2F34A68150442BF23F00705BB
:1012600003F0070343EA4503E3608B6843F0400360
:101270006360CB6843F00103A36042F4967343F0CC
:101280000103236051054FF0FF33236205D512F0AF
:1012900010221DD0B2F1805F1CD080F8643030BDC8
:1012A000104B984208D10E4B1A6C42F480221A64FB
:1012B0001A6E42F48022C5E70B4B9842C4D1084B0A
:1012C0001A6C42F080421A641A6E42F08042B9E70A
:1012D0007F23E2E73F23E0E76C3C0008C8290220B7
:1012E00000380240342A0220A02A022000F1604384
:1012F00000F01F02400903F5614309018000C9B2F3
:1013000000F1604083F8001300F561400123934031
:10131000C0F8803103607047F8B5154682680669E9
:10132000AA420B46816938BF8568761AB5420446E1
:1013300007D218462A46FFF797FDA3692B44A361FD
:101340000DE011D932461846FFF78EFDAF1B3A4625
:10135000E1683044FFF788FDE2683A44A261A3687F
:101360005B1BA3602846F8BD18462A46FFF77CFDA4
:10137000E368E4E783682DE9F041044693421546AB
:10138000266938BF85684069361AB5420F4606D2CD
:101390002A46FFF769FD63692B4463610DE012D9AA
:1013A0003246A5EB0608FFF75FFD4246B919E06833
:1013B000FFF75AFDE26842446261A3685B1BA360C9
:1013C0002846BDE8F0812A46FFF74EFDE368E4E7D2
:1013D00010B50A440024C361029B00604060846031
:1013E000C160816141610261036210BD08B582691B
:1013F0004369934201D1826882B982680132826076
:101400005A1C42611970426903699A4201D3C36848
:101410004361002100F09CFE002008BD4FF0FF302A
:1014200008BD000070B5202304460E4683F31188E2
:10143000A568A5B1A368A269013BA360531CA36181
:1014400015782269934224BFE368A361E3690BB175
:1014500020469847002383F31188284670BD314603
:10146000204600F065FE0028E2DA85F3118870BDA1
:101470002DE9F74F05460F4690469A46D0F81C9046
:10148000202686F311884FF0000B144664B12246E3
:1014900039462846FFF740FF034668B951462846BB
:1014A00000F046FE0028F1D0002383F31188A8EB5A
:1014B000040003B0BDE8F08FB9F1000F03D0019034
:1014C0002846C847019B8BF31188E41A1F4486F312
:1014D0001188DBE7C16081614161C3611144009BF8
:1014E000006040608260016103627047F8B50446A5
:1014F0000E461746202383F31188A568A5B1A3687B
:10150000013BA36063695A1C62611E7023696269B2
:101510009A4224BFE3686361E3690BB120469847B0
:10152000002080F31188F8BD3946204600F000FE07
:101530000028E2DA85F31188F8BD0000836942696A
:101540009A4210B501D182687AB98268013282600C
:101550005A1C82611C7803699A4201D3C368836173
:10156000002100F0F5FD204610BD4FF0FF3010BD0A
:101570002DE9F74F05460F4690469A46D0F81C9045
:10158000202686F311884FF0000B144664B12246E2
:1015900039462846FFF7EEFE034668B9514628460D
:1015A00000F0C6FD0028F1D0002383F31188A8EBDA
:1015B000040003B0BDE8F08FB9F1000F03D0019033
:1015C0002846C847019B8BF31188E41A1F4486F311
:1015D0001188DBE7026843681143016003B11847D3
:1015E000704700001430FFF743BF00004FF0FF3397
:1015F0001430FFF73DBF00003830FFF7B9BF0000DF
:101600004FF0FF333830FFF7B3BF00001430FFF75F
:1016100009BF00004FF0FF311430FFF703BF000097
:101620003830FFF763BF00004FF0FF323830FFF76C
:101630005DBF000000207047FFF774BD044B0360DE
:10164000002343608360C36001230374704700BFBD
:10165000843C000810B52023044683F31188FFF76B
:10166000DDFD02232374002383F3118810BD0000E5
:1016700038B5C36904460D461BB904210844FFF779
:10168000A9FF294604F11400FFF7B0FE002806DA8E
:10169000201D4FF48061BDE83840FFF79BBF38BD87
:1016A000026843681143016003B1184770470000A6
:1016B00013B5446BD4F894341A681178042915D101
:1016C000217C022912D11979128901238B401342FE
:1016D0000CD101A904F14C0001F08EFED4F8944421
:1016E000019B21790246206800F0E0F902B010BDAC
:1016F000143001F011BE00004FF0FF33143001F040
:101700000BBE00004C3001F0E3BE00004FF0FF3391
:101710004C3001F0DDBE0000143001F0DFBD0000F0
:101720004FF0FF31143001F0D9BD00004C3001F012
:10173000AFBE00004FF0FF324C3001F0A9BE0000F8
:10174000D0F8942438B5136819780429054601D0D7
:10175000012038BD017C0229FAD112795C8901206F
:1017600090400440F4D105F1140001F071FD0246EF
:101770000028EDD0D5F894544FF480732868697927
:1017800000F082F9204638BD406BFFF7D9BF00005A
:1017900000207047704700007FB5124B03600023A4
:1017A00043608360C360012502260F4B0574044625
:1017B0000290019300F18402294600964FF4807351
:1017C000143001F021FD094B0193029400964FF46F
:1017D000807304F52372294604F14C0001F0E8FD02
:1017E00004B070BDAC3C000889170008B1160008B1
:1017F0000B68202282F311880A7903EB82021062BF
:101800004A790D3243F822008A7912B103EB820340
:10181000186202230374C0F89414002383F3118820
:101820007047000038B5037F044613B190F8543078
:10183000ABB9201D01250221FFF732FF04F114008E
:1018400025776FF0010100F08FFC84F8545004F10B
:101850004C006FF00101BDE8384000F085BC38BD98
:1018600010B5012104460430FFF71AFF0023237747
:1018700084F8543010BD000038B5044600251430FB
:1018800001F0DAFC04F14C00257701F0A9FD201DE0
:1018900084F854500121FFF703FF2046BDE838408B
:1018A000FFF74EBF90F85C3003F06003202B19D196
:1018B00090F85D20212A0AD0222A4FF000030ED092
:1018C000202A0FD1084A02650722426504E0064B30
:1018D0000365072343650023836501207047036583
:1018E0004365F9E70020704728240220D0F894349B
:1018F00037B51A681178042904461AD1017C0229E7
:1019000017D11979128901238B40134211D100F1AB
:101910004C05284601F024FE58B101A9284601F0E3
:101920006BFDD4F89444019B21790246206800F0B5
:10193000BDF803B030BD000000EB8103F7B51C6AB1
:1019400005460E46F4B1202383F3118805EB860784
:10195000201D0821FFF7A4FEFB685B691B684C345F
:1019600013B1204601F056FD01A9204601F044FDC7
:10197000024648B1019B3146284600F097F8002303
:1019800083F3118803B0F0BDFB685A691268002A1E
:10199000F5D01B8A013B1340F1D105F15C02EAE767
:1019A0000D3138B550F82140DCB1202383F3118884
:1019B000D4F894241368527903EB8203DB689B69A3
:1019C0005D6845B104216018FFF76AFE294604F1FD
:1019D000140001F047FC2046FFF7B2FE002383F31A
:1019E000118838BD7047000000F0F4BF0123037078
:1019F0000023436000F1240200F1380142F8043B67
:101A00008A421361FAD103814381704738B5044695
:101A1000202383F3118800254160C560056145617D
:101A20008561C561056200F0E5FF0223237085F33F
:101A3000118838BD70B500EB810305465069DA6046
:101A40000E46144618B110220021FFF737FAA0699C
:101A500018B110220021FFF731FA31462846BDE8BF
:101A6000704001F091B80000028902F00102028189
:101A7000428902F0010242810022026142618261D8
:101A8000C261026201F014B9F0B400EB810447892D
:101A9000E4680125A4698D403D434581236000230E
:101AA000A2606360F0BC01F02FB90000F0B400EB5D
:101AB00081040789E468012564698D403D430581FF
:101AC00023600023A2606360F0BC01F0A9B90000AC
:101AD00070B50223002504460370A0F8645080F816
:101AE000665080F8675005814581C5600561456194
:101AF0008561C561056280F84C5000F0E1FF6368C4
:101B00001B6823B129462046BDE87040184770BDC8
:101B1000436802781B6880F86820052202700BB1C8
:101B20000421184770470000436890F868201B683C
:101B300002700BB1052118477047000090F84C3037
:101B400070B5044613B1002380F84C3004F15C02F8
:101B5000204601F0CFF863689B6863BB94F85C5043
:101B600015F0600615D194F85D3005F07F0545EA63
:101B7000032540F202339D4200F00E815BD8022D16
:101B800000F0DC803FD8002D00F08780012D00F0B0
:101B9000CF800021204601F019FB0021204601F0F2
:101BA0000BFB63681B6813B1062120469847062388
:101BB00084F84C3070BD204698470028CED094F869
:101BC000632094F8623043EA0223626D934238BF87
:101BD000636594F95C30656D002B4FF0200380F253
:101BE000FD80002D00F0EC80092284F84C2083F366
:101BF00011880021636D226D2046FFF757FF0023F7
:101C000083F3118870BDB5F5817F00F0B180B5F523
:101C1000407F49D0B5F5807FBBD194F85E30012B71
:101C2000B7D1B4F8643023F00203A4F86430266519
:101C30006665A665C3E740F201639D421ED8B5F50F
:101C4000C06F3BD2B5F5A06FA3D1B4F85C30B3F54B
:101C5000A06F0ED194F85E3084F86630204600F014
:101C600087FF63681B6813B101212046984703234F
:101C70002370002323656365A365A0E7B5F5106FA6
:101C800032D040F602439D4252D0B5F5006F80D16C
:101C900004F167032365012324E004F16403236551
:101CA00002236365A5658AE794F85E30012B7FF413
:101CB00070AFB4F8643043F00203B6E794F86120E3
:101CC000616894F860304D6894F85F1043EA02232D
:101CD000204694F85E20A84700283FF45AAF436896
:101CE000236503686365A4E72378042B10D12023C0
:101CF00083F311882046FFF7B7FE86F311886368E7
:101D000084F867601B68032121700BB12046984757
:101D100094F85E30002BACD084F867300423237035
:101D200063681B68002BA4D0022120469847A0E7D7
:101D3000374B23650223636500239DE794F8601009
:101D400011F0800F204601F00F010ED000F0C4FF0B
:101D5000012806D002287FF41CAF2E4B2365606556
:101D600067E72D4B2365656563E700F0A7FFEFE7A5
:101D700094F85E30002B7FF40CAF94F8603013F0D1
:101D80000F013FF476AF1A06204602D501F032FA71
:101D90006FE701F025FA6CE794F85E30002B7FF4D2
:101DA000F8AE94F8603013F00F013FF462AF1B06F9
:101DB000204602D501F00AFA5BE701F0FDF958E789
:101DC000142284F84C2083F311882B462A46294696
:101DD0002046FFF759FE85F3118870BD5DB11522CD
:101DE00084F84C2083F311880021636D226D204616
:101DF000FFF74AFE03E70B2284F84C2083F3118897
:101E00002B462A4629462046FFF750FEE3E700BF4F
:101E1000DC3C0008D43C0008D83C000838B590F8F9
:101E20004C300446152B29D8DFE803F03E2828283B
:101E300028283E28280B2939282828282828282817
:101E40003E3E90F8631090F86220436D42EA012212
:101E50009A4214D9C268128AB3FBF2F502FB153517
:101E60006DB9202383F311882B462A462946FFF7B4
:101E70001DFE85F311880A2384F84C3038BD1423E5
:101E800084F84C30202383F3118800231A46194626
:101E90002046FFF7F9FD002383F3118838BD836DD9
:101EA00003B198470023E7E7002101F08FF90021F3
:101EB000204601F081F963681B6813B106212046B2
:101EC00098470623D8E7000090F84C20152A38B52B
:101ED000044622D80123934040F6416213421DD1AB
:101EE00013F480150FD19B0217D50B2380F84C30CB
:101EF000202383F311882B462A462946FFF7D6FD77
:101F000085F3118838BDC3689B695B682BB9836D05
:101F100003B19847002384F84C3038BD002101F00C
:101F200055F90021204601F047F963681B6813B199
:101F30000621204698470623EDE70000024B0022C9
:101F40001B605B609A6070470C37022000230374AB
:101F50008268054B1B6899689142FBD25A680360FE
:101F600042601060586070470C37022008B520238B
:101F700083F31188037C032B05D0042B0DD02BB9E0
:101F800083F3118808BD436900221A604FF0FF33C4
:101F90004361FFF7DBFF0023F2E790E80C001A60D3
:101FA00002685360F2E70000002303748268054B67
:101FB0001B6899689142FBD85A68036042601060C0
:101FC000586070470C370220054B1969087418686F
:101FD00002681A605360186101230374FEF7A4B904
:101FE0000C37022030B54B1C87B005460A4C10D088
:101FF00023690A4A01A800F0D3F82846FFF7E4FF56
:10200000049B13B101A800F007F92369586907B0D0
:1020100030BDFFF7D9FFF8E70C3702206D1F00082D
:1020200038B50C4D41612B6981689A68914204462C
:1020300003D8BDE83840FFF789BF1846FFF786FF91
:1020400001232C61014623742046BDE83840FEF789
:102050006BB900BF0C370220044B1A681B699068EB
:102060009B68984294BF0020012070470C370220E3
:1020700010B5084C236820691A6822605460012258
:1020800023611A74FFF790FF01462069BDE81040F4
:10209000FEF74AB90C370220826002220274002245
:1020A000427470478368A3F17C0243F80C2C0269E8
:1020B00043F83C2C426943F8382C074A43F81C2C5F
:1020C000C26843F8102C022203F8082C002203F8FF
:1020D000072CA3F1180070474103000810B5202316
:1020E00083F31188FFF7DEFF00210446FFF798FF16
:1020F000002383F31188204610BD0000024B1B69AA
:1021000058610F20FFF760BF0C370220202383F3B4
:102110001188FFF7F3BF000008B50146202383F3C1
:1021200011880820FFF75EFF002383F3118808BDA4
:1021300049B1064B42681B6918605A6013604360DE
:102140000420FFF74FBF4FF0FF3070470C370220DD
:102150000368984206D01A680260506059611846B8
:10216000FFF7F4BE7047000038B504460D462068FE
:10217000844200D138BD036823605C604561FFF78D
:10218000E5FEF4E7054B03F114025A619A614FF042
:10219000FF32DA6100221A62704700BF0C3702205A
:1021A000F8B503614FF08043C2605C6A194B1A4670
:1021B000022952F8145F38BF0221954206461F4695
:1021C0000AD1586198611C620560456081600819F8
:1021D000BDE8F84001F0E6B9186AAB68241A0C199A
:1021E00002D3E41A2D6804E09C4202D2204401F09C
:1021F000E7F9AB689C42F4D86B68736035601E6089
:102200006E60B460A9684FF0FF33091BA960FB61E1
:10221000F8BD00BF0C37022010B41B4C234653F806
:10222000141F814210D0416802680A600268516040
:102230009A424FF00001C16003D0936881680B445B
:1022400093605DF8044B70470A68626100209A420F
:102250005360C86003D15DF8044B01F0ABB99368DB
:102260008868034493604FF08042206A526A121AD1
:102270009342E6D9991A012998BF931C18445DF836
:10228000044B01F09DB900BF0C37022000207047BD
:10229000FEE70000704700004FF0FF30704700007D
:1022A000022906D0032906D00129064818BF0020BC
:1022B000704705487047032A9ABF044800EBC200E4
:1022C00000207047CC3D0008803D000830240220EB
:1022D00070B5044608460D46FEF7E8FDC6B2204636
:1022E000013403780BB9184670BD32462946FEF713
:1022F000C5FD0028F3D1012070BD00002DE9F04F8D
:1023000081469BB008460C461646FEF7CFFD3C4979
:10231000C5B22046FFF7DCFF08B10335EDB23949FD
:102320002046FFF7D5FF08B11035EDB2632D01AFA0
:102330000CD8DFF8DCA0DFF8DCB03D4694F8008074
:10234000B8F1000F1CD185F8008003E02146384623
:1023500001F05EFC3846FEF7A9FDC0B2431C5B00ED
:1023600089E848003370032373700023023619464E
:10237000DAB2904206F102063AD81BB0BDE8F08FFF
:10238000B8F1250F2FD107221D492046FEF776FD13
:1023900058B9DBF800202A60DBF804206A60BBF83B
:1023A00008202A8107340A35C8E708221549204643
:1023B000FEF764FDB8B91448AA1C10F8011F134BAE
:1023C0004FEA111E01F00F011EF80AE011F80A1081
:1023D00002F802EC984202F8011C02F10202ECD170
:1023E00018350834AAE785F8008001340135A5E7DF
:1023F000FA5C06F8022C06F8011C0133B8E700BFAE
:10240000303D0008383D00081FF4F01F2BF4F01F8A
:102410004C3D0008413D000808B5202383F3118896
:102420000348FFF763FA002383F3118808BD00BF58
:102430004C37022010B50446052916D8DFE801F014
:1024400016150316161D202383F311880E4A012149
:10245000FFF7F0FA20460D4A0221FFF7EBFA0C488D
:10246000FFF70AFA002383F3118810BD202383F3BA
:1024700011880748FFF7D6F9F4E7202383F3118882
:102480000348FFF7EDF9EDE7E03C0008043D0008E4
:102490004C37022038B50C4D0C4C0D492A4604F13E
:1024A0000800FFF72BFF05F1CA0204F110000949EB
:1024B000FFF724FF05F5CA7204F118000649BDE8CC
:1024C0003840FFF71BBF00BF143C0220302402201D
:1024D000603D0008643D0008383D0008BFF34F8FA1
:1024E000024AD368DB03FCD4704700BF003C0240C3
:1024F00008B5074B1B7853B9FFF7F0FF054B1A6976
:10250000002ABFBF044A5A6002F188325A6008BDEF
:10251000723E0220003C02402301674508B5054B8E
:102520001B7833B9FFF7DAFF034A136943F000431E
:10253000136108BD723E0220003C02400B2870B5BA
:1025400013D80B4A0B4C137863B90B4E4FF0006154
:1025500044F8231056F8235001330C2B2944F7D1AB
:102560000123137054F8200070BD002070BD00BF1F
:10257000A43E0220743E0220EC3D0008014B53F8BB
:1025800020007047EC3D00080C2070470B2810B568
:10259000044601D9002010BDFFF7D0FF064B53F8C9
:1025A00024301844C21A0BB9012010BD1268013240
:1025B000F0D1043BF6E700BFEC3D00080B2810B556
:1025C00004462FD8FFF78AFFFFF792FF1649F3233F
:1025D000CB60FFF783FFC300DBB243F4007343F02B
:1025E00002030B610B6943F480330B61FFF776FF45
:1025F000FFF7A4FF0D4B53F824300344BFF34F8F74
:102600000B4A98420AD3BFF34F8FBFF36F8FFFF788
:1026100085FF2046BDE81040FFF7B8BFC2F85C0256
:102620002030EEE7002010BD003C0240EC3D0008E9
:1026300000ED00E02DE9F84312F00103154643D107
:102640000244B2F1026F3FD22C4B1B6813F001031E
:102650003AD02B4CFFF74CFFF323E360FFF73EFF2C
:1026600040F20127032D16D8254C0F46401A40F2A0
:102670000118EB1B0B44012B00EB0706236926D83E
:1026800023F001032361FFF749FF0120BDE8F88330
:10269000043D0430E6E78307E6D1236923F4407361
:1026A000236123693B43236151F8046B0660BFF348
:1026B0004F8FFFF713FF03689E42E9D0236923F091
:1026C00001032361FFF72AFF0020BDE8F88323F40C
:1026D00040732361236943EA08032361B94637F84D
:1026E000023B3380BFF34F8FFFF7F8FE3688B9F80F
:1026F0000030B6B2B342BCD0E0E700BF00380240C1
:10270000003C0240084908B50B7828B153B9FFF7DF
:10271000EFFE01230B7008BD23B1BDE8084008702F
:10272000FFF7FCBE08BD00BF723E0220014B53F80C
:1027300020007047502800400A4B1A6F120407D43B
:102740001A6F42F400721A671A6F42F400421A6755
:10275000054A136843F48073136000B2034B43F8D7
:1027600020107047003802400070004050280040A0
:10277000014B1868704700BF5028004001460020F8
:10278000FFF7DABF38B5094B1B689B000CD5084B27
:10279000084D01221A700024E0B2FFF7C7FF45F888
:1027A00024000134082CF7D138BD00BF7438024032
:1027B000C83E0220A83E0220014B1878704700BF97
:1027C000C83E0220064A536823F001035360EFF32A
:1027D0000983683383F30988002383F311887047E2
:1027E00030EF00E010B5202383F31188104B5B68B5
:1027F00013F4006318D0F1EE103AEFF309844FF0B0
:10280000807344F84C3C0B4BDB6844F8083CA4F163
:10281000680383F30988FFF71FFC18B1064B44F8DF
:10282000503C10BD054BFAE783F3118810BD00BF83
:1028300000ED00E030EF00E0510300085403000811
:10284000F0B5BFF34F8FBFF36F8F1D4B0021C3F85F
:102850005012BFF34F8FBFF36F8F5A6942F40032AB
:102860005A61BFF34F8FBFF36F8FC3F88410BFF36C
:102870004F8FD3F88020C2F3C904C2F34E32520105
:10288000A50743F6E07602EA060E284621464EEA00
:1028900000070139C3F860724F1C00F14040F6D1C7
:1028A000203A12F1200FEED1BFF34F8F5A6942F454
:1028B00080325A61BFF34F8FBFF36F8FF0BD00BFFF
:1028C00000ED00E0FEE70000084A094B09498B4291
:1028D00004D3094A0021934205D3704752F8040FEC
:1028E00043F8040BF3E743F8041BF4E7F43F000854
:1028F000D8410220D8410220D8410220036F30B5D0
:1029000000229D68C46E11464FF0FF3004EB421365
:1029100001329542C3F80019C3F81019C3F8080929
:10292000C3F8001BC3F8101BC3F8080BEED24FF01E
:102930000113C4F81C3830BD890141F02001016148
:1029400003699B06FCD4122000F0C8BE204B03EBA9
:1029500080022DE9F047D2F80CE0DD6EDEF814209D
:10296000461CD2F800C005EB063605EB401851684E
:1029700061450BD3D5F83428012303FA00F022EA8D
:102980000000C5F834081846BDE8F087BEF81040CE
:10299000ACEB0103A34228BF2346D8F81849A4B2E0
:1029A000B3EB840F10D894681F46A4F1040959F8BA
:1029B00004AFC6F800A0042F01D9043FF7E71C4478
:1029C0000B4494605360D2E70020BDE8F08700BF5D
:1029D000CC3E022010B5054C2046FFF707F84FF01B
:1029E000A043E366024B236710BD00BFCC3E02202C
:1029F000403E00080378012B70B5054650D12A4BA4
:102A0000C46E98421BD1294B5A6B42F080025A6324
:102A10005A6D42F080025A655A6D5A6942F080023E
:102A20005A615A6922F080025A610E2143205B6983
:102A3000FEF75CFC1E4BE3601E4BC4F8003800231D
:102A4000C4F8003EC0232360EE6E4FF40413A3636A
:102A50003369002BFCDA012333610C2000F03EFEC9
:102A60003369DB07FCD4122000F038FE3369002BF9
:102A7000FCDA0026A6602846FFF740FF6B68C4F822
:102A80001068DB68C4F81468C4F81C684BB90A4BBA
:102A9000A3614FF0FF336361A36843F00103A360B8
:102AA00070BD064BF4E700BFCC3E02200038024068
:102AB0004014004003002002003C30C0083C30C0FD
:102AC000F8B5C46E054600212046FFF735FF296F93
:102AD00000234FF001128F68C4F834384FF00066BD
:102AE000C4F81C284FF0FF3004EB431201339F421F
:102AF000C2F80069C2F8006BC2F80809C2F8080BF6
:102B0000F2D20B68EA6E6B67636210231361166979
:102B100016F01006FBD1122000F0E0FDD4F80038CA
:102B200023F4FE63C4F80038A36943F4402343F060
:102B30001003A3610923C4F81038C4F814380A4BF1
:102B4000EB604FF0C043C4F8103B084BC4F8003BA7
:102B5000C4F81069C4F800396B6F03F1100243F434
:102B600080136A67A362F8BD1C3E00084080001015
:102B7000C26E90F86610D2F8003823F4FE6343EA80
:102B80000113C2F8003870472DE9F0410EB200EB96
:102B900086080D46D8F80C100F6807F00303022BC7
:102BA00050D0032B50D03D4A3D4F012B18BF174644
:102BB000C46E4FEA451E04EB0E030022C3F8102B2F
:102BC0008A6905F1100C002A40D04A8A05F15803A1
:102BD0005B013A43E2500123D4F81C2803FA0CF3BA
:102BE0001343A6444A69C4F81C380023CEF81039B0
:102BF00005F13F03002A39D00A8A898B92080129FE
:102C000088BF4A43416F04EB8303561841EA0242EE
:102C1000466729465A602046FFF78EFED8F80C30EA
:102C20001B8A43EA85531F4305F148035B01E750C4
:102C30000123D4F81C2803FA05F51543C4F81C58E1
:102C4000BDE8F081174FB3E7174FB1E704EB461328
:102C5000D3F8002B22F40042C3F8002BD4F81C2830
:102C6000012303FA0CF322EA0303BAE704EB83031C
:102C70000E4A5A6004EB461629462046FFF75CFED2
:102C8000D6F8003923F40043C6F80039D4F81C38CC
:102C9000012202FA05F523EA0505CFE700800010BE
:102CA000008004100080081000800C100004000256
:102CB000026F12684267FFF721BE00005831C36EF1
:102CC00049015B5813F4004004D013F4001F14BFF3
:102CD00001200220704700004831C36E49015B5853
:102CE00013F4004004D013F4001F14BF012002208D
:102CF0007047000000EB8101CB68196A0B68136014
:102D00004B6853607047000000EB810330B5DD680D
:102D1000AA691368D36019B9402B84BF402313609C
:102D20006B8A1468C26E1C44013CB4FBF3F4634329
:102D3000033323F0030302EB411043EAC44343F09F
:102D4000C043C0F8103B2B6803F00303012B09B20A
:102D50000ED1D2F8083802EB411013F4807FD0F87E
:102D6000003B14BF43F0805343F00053C0F8003BD6
:102D700002EB4112D2F8003B43F00443C2F8003B9F
:102D800030BD00002DE9F041244DEE6E06EB4013FE
:102D90000446D3F8087BC3F8087B38070AD5D6F871
:102DA0001438190706D505EB84032146DB6828464D
:102DB0005B689847FA072FD5D6F81438DB072BD570
:102DC00005EB8403D968CCB98B69488A5E68B6FB89
:102DD000F0F200FB12628AB91868DA6890420DD2EC
:102DE000121A83E81400202383F311880B4821462C
:102DF000FFF78AFF84F31188BDE8F081012303FA0D
:102E000004F26B8923EA02036B81CB6823B121466C
:102E10000248BDE8F0411847BDE8F081CC3E0220F1
:102E200000EB810370B5DD68C36E6C692668E660EF
:102E30004A0156BB1A444FF40020C2F810092A6810
:102E400002F00302012A0AB20ED1D3F8080803EBFC
:102E5000421410F4807FD4F8000914BF40F0805071
:102E600040F00050C4F8000903EB4212D2F8000908
:102E700040F00440C2F80009D3F83408012202FAF5
:102E800001F10143C3F8341870BD19B9402E84BF55
:102E90004020206020682E8A841940F00050013CB8
:102EA0001A44B4FBF6F440EAC440C6E7F8B5044659
:102EB0001E48C56E05EB4413D3F80869C3F80869CA
:102EC000F10717D5D5F81038DA0713D500EB8403CE
:102ED000D9684B691F68DA68974218D2D21B00275D
:102EE0001A605F60202383F311882146FFF798FF63
:102EF00087F31188330617D5D5F834280123A3406A
:102F0000134211D02046BDE8F840FFF71FBD012352
:102F100003FA04F2038923EA020303818B68002B7E
:102F2000E8D021469847E5E7F8BD00BFCC3E022037
:102F3000A0482DE9F84FC56E6E69AB691E4016F4C6
:102F4000805F6E61044605D0FEF7C2FDBDE8F84F14
:102F5000FFF748BC002E12DAD5F8003E95489B07D3
:102F60001EBFD5F8003E23F00303C5F8003ED5F898
:102F7000043823F00103C5F80438FEF7D5FD370502
:102F800002D58C48FEF7C4FDB0040CD5D5F808383E
:102F900013F0060FEB6823F470530CBF43F4105387
:102FA00043F4A053EB60310704D56368DB680BB1D1
:102FB00080489847F2026FD4B3020CD5D4F86C80E5
:102FC000DFF8F0A100274FF00109236F9B68F9B2E9
:102FD0008B4280F09C80F70619D5E16E0A6AC2F335
:102FE0000A1702F00F0302F4F012B2F5802F00F07E
:102FF000B680B2F5402F0AD104EB830301F580516E
:10300000DB68186A00231A469F4240F09C80330315
:10301000D5F818481DD5E70302D50020FFF7B2FE0A
:10302000A50302D50120FFF7ADFE600302D5022003
:10303000FFF7A8FE210302D50320FFF7A3FEE2025B
:1030400002D50420FFF79EFEA30202D50520FFF75C
:1030500099FE77037FF57AAFE60702D50020FFF7E8
:1030600025FFA50702D50120FFF720FF600702D545
:103070000220FFF71BFF210702D50320FFF716FFF1
:10308000E20602D50420FFF711FFA3067FF55EAF2D
:103090000520FFF70BFF59E7D4F86C80DFF814A187
:1030A00000274FF00109236F9B685FFA87FB5B45A0
:1030B00082D308EB4B13D3F8002902F44022B2F577
:1030C000802F22D1D3F80029002A1EDAD3F8002954
:1030D00042F09042C3F80029D3F80029002AFBDB14
:1030E0005946E06EFFF728FC228909FA0BF322EA21
:1030F0000303238104EB8B03DB689B6813B1594600
:10310000504698475846FFF721FC0137CBE708EBBC
:103110004112D2F8003B03F44023B3F5802F10D1C5
:10312000D2F8003B002B0CDA628909FA01F322EA9B
:103130000303638104EB8103DB68DB680BB150465A
:103140009847013741E79C0708BF0A68072B98BFDB
:10315000027003F101039CBF120A013054E70233ED
:1031600004EB830201F58051526890690268D0F83F
:1031700008C04068A2EB000E0022104697420AD118
:1031800004EB830463689B699A683A449A605A68BE
:1031900017445F603BE712F0030F08BF08689645CD
:1031A00088BF8CF8000002F1010284BF000A0CF114
:1031B000010CE3E7CC3E0220C36E03EB4111D1F8D2
:1031C000003B43F40013C1F8003B7047C36E03EBB0
:1031D0004111D1F8003943F40013C1F800397047A8
:1031E000C36E03EB4111D1F8003B23F40013C1F887
:1031F000003B7047C36E03EB4111D1F8003923F453
:103200000013C1F80039704730B5039C01720433D4
:1032100004FB0325C361049B03630021059B00603D
:103220004060C16042610261856104624262816204
:10323000C162436330BD00000022416A4161016107
:10324000C2608262C2626FF00101FEF78DBF0000B2
:1032500003694269934203D1C2680AB100207047F2
:10326000181D704703691960C2680132C260C269E3
:10327000134482690361934224BF436A03610021BE
:10328000FEF766BF38B504460D46E3683BB1626998
:10329000131D1268A3621344E362002038BD237A31
:1032A00033B929462046FEF743FF0028EDDA38BD42
:1032B0006FF00100FBE70000C368C269013BC36017
:1032C0004369134482694361934224BF436A436163
:1032D00000238362036B03B11847704770B5202346
:1032E000044683F31188866A3EB9FFF7CBFF054693
:1032F00018B186F31188284670BDA36AE26A13F8F4
:10330000015BA362934202D32046FFF7D5FF00235F
:1033100083F31188EFE700002DE9F84F04460E46CD
:1033200090469946202787F311880025AA46D4F8AD
:1033300028B0BBF1000F09D149462046FFF7A2FF94
:1033400020B18BF311882846BDE8F88FA16AE36AA3
:10335000A8EB050B5B1A9B4528BF9B46BBF1400FB2
:103360001BD9334601F1400251F8040B43F8040B1A
:103370009142F9D1A36A40334036A3624035A26A34
:10338000E36A9A4202D32046FFF796FF8AF3118838
:103390004545D8D287F31188C9E730465A46FDF72C
:1033A00063FDA36A5B445E44A3625D44E7E70000FB
:1033B00010B5029C0172043303FB0421C361002396
:1033C0008362C362039B0363049B00604060C4602C
:1033D00042610261816104624262436310BD000088
:1033E000026AC260426A4261026100228262C26273
:1033F0006FF00101FEF7B8BE436902699A4203D13A
:10340000C2680AB100207047184650F8043B0B60B0
:1034100070470000C368C2690133C3604369134445
:1034200082694361934224BF436A43610021FEF7EE
:103430008FBE000038B504460D46E3683BB12369F2
:103440001A1DA262E2691344E362002038BD237AA8
:1034500033B929462046FEF76BFE0028EDDA38BD69
:103460006FF00100FBE7000003691960C268013AD0
:10347000C260C269134482690361934224BF436AF4
:10348000036100238362036B03B118477047000098
:1034900070B5202304460E4683F31188856A35B93A
:1034A0001146FFF7C7FF10B185F3118870BDA36AFD
:1034B0001E70A36AE26A01339342A36204D3E169F6
:1034C00020460439FFF7D0FF002080F3118870BD3B
:1034D0002DE9F84F04460D4691469A464FF02008D4
:1034E00088F311880026B346A76A4FB95146204693
:1034F000FFF7A0FF20B187F311883046BDE8F88FB1
:10350000A06AE76AA9EB06033F1A9F4228BF1F463D
:10351000402F1BD905F1400355F8042B40F8042B2C
:103520009D42F9D1A36A4033A3624036A26AE36A9E
:103530009A4204D3E16920460439FFF795FF8BF3E3
:1035400011884E45D9D288F31188CDE729463A46ED
:10355000FDF78AFCA36A3B443D44A3623E44E5E791
:10356000026943699A4203D1C3681BB91846704780
:103570000023FBE7836A002BF8D0043B9B1AF5D0AD
:103580001360C368013BC360C3691A448369026165
:103590009A4224BF436A0361002383620123E5E763
:1035A00000F042B94FF08043002258631A610222B2
:1035B000DA6070474FF080430022DA607047000005
:1035C0004FF0804358637047FEE7000010B5194C78
:1035D000FEF7B4FCFEF7D6FD802217492046FEF721
:1035E0005BFD012344F8180C0374144B144AD9688A
:1035F00021F4E0610904090C0A431249DA60CA683F
:1036000042F08072CA60104A1049C2F8B01F1168B7
:1036100041F0010111601022DA77202283F8222084
:10362000002383F3118862B60948BDE81040FEF715
:1036300055BD00BF343702204C3E000800ED00E0CD
:103640000003FA05F0ED00E0001000E055CEACC537
:10365000543E00082DE9F84F1F4C4FF000086569F3
:1036600004F11407C1464FF08043266A5B6AAA68DA
:103670009E1B96421DD34FF0200AAA68236AD5F8F4
:103680000CB0134423622B68BB425F60A6EB0206BA
:103690006361C5F80C8001D1FFF78CFF89F31188B5
:1036A0002869D8478AF311886569AB689E42E4D2DD
:1036B000D9E76269BA420CD0916823628E1B96608A
:1036C000A86802282CBF1818981CBDE8F84FFFF70F
:1036D00077BFBDE8F88F00BF0C370220034B596855
:1036E0005A68521A9042FBD8704700BF001000E0A1
:1036F0004B6843608B688360CB68C3600B69436130
:103700004B6903628B6943620B680360704700007A
:1037100008B5274B27481A6940F2FF710A431A611E
:103720001A6922F4FF6222F007021A611A691A6B01
:103730000A431A631A6D0A431A651F4A1B6D114624
:10374000FFF7D6FF1D4802F11C01FFF7D1FF1C480F
:1037500002F13801FFF7CCFF1A4802F15401FFF7DC
:10376000C7FF194802F17001FFF7C2FF174802F1C5
:103770008C01FFF7BDFF164802F1A801FFF7B8FF63
:10378000144802F1C401FFF7B3FF134802F1E0014E
:10379000FFF7AEFF114802F1FC01FFF7A9FF104847
:1037A00002F58C71FFF7A4FFBDE8084000F09EB859
:1037B0000038024000000240743E0008000402404D
:1037C00000080240000C02400010024000140240B9
:1037D00000180240001C0240002002400024024069
:1037E0000028024008B500F0F5F9FFF7EFFEFEF7FC
:1037F000C9FFBDE80840FEF74DBE0000704700005D
:103800004FF0804310B51A69920708D500241C6157
:10381000202383F31188FFF71DFF84F31188BDE88F
:103820001040FEF7DFBF0000104B1A6C42F001029F
:103830001A641A6E42F001021A660D4A1B6E9368F2
:1038400043F0010393604FF080436B229A624FF084
:10385000FF32DA6200229A615A63DA605A6001220A
:103860005A6108211A601C20FDF740BD0038024053
:10387000002004E01B4B1A696FEA42526FEA525271
:103880001A611A69C2F30A021A614FF0FF301A690D
:103890005A69586100215A6959615A691A6A62F075
:1038A00080521A621A6A02F080521A621A6A5A6ABE
:1038B00058625A6A59625A6A0B4A106840F480701A
:1038C0001060186F00F44070B0F5007F1EBF4FF419
:1038D000803018671967536823F40073536000F051
:1038E00059B900BF0038024000700040354B364ADD
:1038F0001A64364A4FF4404111601A6842F00102DE
:103900001A601A689207FCD59A6822F003029A603E
:103910002C4B19469A6812F00C02FBD1186800F083
:10392000F90018609A601A6842F480321A600B68D5
:103930009B03FCD54B6F43F001034B67214B5A6F40
:103940009007FCD5224A5A601A6842F080721A60C9
:103950001E4B1A4659684904FCD5196841F4803158
:1039600019605368D803FCD5136843F4003313601F
:10397000164A53689903FCD5124B1A689201FCD57C
:10398000144A9A6040F20112C3F88C200022C3F856
:103990009020114A40F2073111609A6842F0020209
:1039A0009A60084B9A6802F00C02082AFAD15A6C05
:1039B00042F480425A645A6E42F480425A665B6E08
:1039C000704700BF00380240000400100070004043
:1039D000186C400900948838003C0240084A08B539
:1039E000536911680B4003F00103536123B1054A89
:1039F00013680BB150689847BDE80840FEF7F2BE67
:103A0000003C014058410220084A08B5536911683A
:103A10000B4003F00203536123B1054A93680BB1D5
:103A2000D0689847BDE80840FEF7DCBE003C014086
:103A300058410220084A08B5536911680B4003F049
:103A40000403536123B1054A13690BB150699847C8
:103A5000BDE80840FEF7C6BE003C014058410220C8
:103A6000084A08B5536911680B4003F00803536115
:103A700023B1054A93690BB1D0699847BDE8084066
:103A8000FEF7B0BE003C014058410220084A08B58C
:103A9000536911680B4003F01003536123B1054AC9
:103AA000136A0BB1506A9847BDE80840FEF79ABE0A
:103AB000003C014058410220174B10B55C691A6860
:103AC000144004F478725A61A30604D5134A936A29
:103AD0000BB1D06A9847600604D5104A136B0BB13E
:103AE000506B9847210604D50C4A936B0BB1D06BF1
:103AF0009847E20504D5094A136C0BB1506C9847FE
:103B0000A30504D5054A936C0BB1D06C9847BDE86A
:103B10001040FEF767BE00BF003C01405841022044
:103B20001A4B10B55C691A68144004F47C425A615F
:103B3000620504D5164A136D0BB1506D98472305E5
:103B400004D5134A936D0BB1D06D9847E00404D5AA
:103B50000F4A136E0BB1506E9847A10404D50C4A5E
:103B6000936E0BB1D06E9847620404D5084A136F68
:103B70000BB1506F9847230404D5054A936F0BB1DE
:103B8000D06F9847BDE81040FEF72CBE003C0140C6
:103B900058410220062108B50846FDF7A7FB06217B
:103BA0000720FDF7A3FB06210820FDF79FFB062158
:103BB0000920FDF79BFB06210A20FDF797FB062154
:103BC0001720FDF793FB06212820BDE80840FDF7EC
:103BD0008DBB000008B5FFF74DFE00F00DF8FDF7B6
:103BE0002BFDFDF701FFFDF7D5FDFFF707FEBDE853
:103BF0000840FFF7D5BC0000002304491A465A507C
:103C0000C8180833802B4260F9D170475841022010
:103C1000034611F8012B03F8012B002AF9D1704754
:103C200012101213121100000010410001105A006E
:103C30004C370220C8290220342A0220A02A022060
:103C400053544D3332463F3F3F3F3F3F0053544D67
:103C5000333246375B347C355D780053544D333214
:103C600046375B367C375D78000000000096000028
:103C70000000000000000000000000000000000044
:103C8000000000000000000001160008ED1500080B
:103C90002916000815160008211600080D16000840
:103CA000F9150008E51500083516000800000000A9
:103CB0000D170008F916000835170008211700082D
:103CC0002D1700081917000805170008F11600083D
:103CD0009117000800000000010000000000000033
:103CE000020000000000000039190008A1190008B6
:103CF00040004000E43B0220F43B022002000000B0
:103D0000000000000300000000000000E5190008AA
:103D10000000000010000000043C02200000000031
:103D20000100000000000000CC3E02200101020062
:103D300025424F41524425002553455249414C25C7
:103D4000006D526F5832312D3737370030313233F2
:103D50003435363738394142434445460000000087
:103D60006D526F0058322E312D373737000000006A
:103D700035240008A1220008A5180008192400080D
:103D800043000000883D000809024300020100C012
:103D9000320904000001020201000524001001059F
:103DA0002401000104240202052406000107058203
:103DB000030800FF09040100020A000000070501D2
:103DC00002400000070581024000000012000000D0
:103DD000D43D000812011001020000408304405746
:103DE0000002010203010000040309040080000036
:103DF0000080000000800000008000000000020041
:103E000000000400000004000000040000000400A2
:103E10000000040000000400000004000000000096
:103E20003D1B00081D1E0008C91E00084000400080
:103E3000443F0220443F022001000000543F022082
:103E40008000000040010000050000006D61696E07
:103E5000000000006C3E0008603F02205841022034
:103E600001000000C93500080000000069646C65AD
:103E7000000000000000802A00000000AAAAAAAAF0
:103E800000000000FFFF00000000000000A00A008A
:103E90000000000000000000AAAAAAAA000000007A
:103EA000FFFF000000000000000000000000000014
:103EB00000000000AAAAAAAA00000000FFFF00005C
:103EC000000000000000000080298A0100000000BE
:103ED000AAAAAAAA40154501FFFF000000707007BA
:103EE000777000000080020100000000AAAAAAAAC0
:103EF00000400100FFFF00000000008008000000FB
:103F00000000000000000000AAAAAAAA0000000009
:103F1000FFFF0000000000000000000000000000A3
:103F200000000000AAAAAAAA00000000FFFF0000EB
:103F30000000000000000000000000000000000081
:103F4000AAAAAAAA00000000FFFF000000000000CB
:103F5000000000000000000000000000AAAAAAAAB9
:103F600000000000FFFF0000000000000000000053
:103F70000000000000000000000000000000000041
:103F80000000000000000000000000000000000031
:103F90000000000000000000000000000000000021
:103FA0000000000000000000FF0000000000000012
:103FB000403C00083F000000490400004D3C000860
:103FC0003F000000510400005B3C00083F0000007F
:103FD000009600000000080004000000E83D000812
:103FE00000000000000000000000000000000000D1
:083FF0000000000000000000C9
:00000001FF
